:100000000C94A0020C9450240C94BD020C94BD02DC
:100010000C94BD020C94BD020C94BD020C94BD0264
:100020000C94BD020C94BD020C946F2B0C94412CCB
:100030000C945A260C94BD020C94BD020C94BD0283
:100040000C94BD020C94BD020C94BD020C94BD0234
:100050000C94BD020C94FE260C94BD020C94BD02BF
:100060000C94BD020C94BD020C94BD020C94BD0214
:100070000C94BD020C94BD020C94BD020C94BD0204
:100080000C94BD020C94BD020C94BD020C94BD02F4
:100090000C94BD020C94BD020C94BD020C94BD02E4
:1000A0000C94BD020C94BD020C94BD029205920505
:1000B000BE05BE05260644065C075C074F06E8063B
:1000C000F906F906AE2CD52CCD2DD52CCD2D212D14
:1000D000442DCD2D9B2DAA2D165C1E001F00200047
:1000E0002100220000002B0014001A000800150057
:1000F00017000000394104001600070009000A003B
:100100000000E1001D001B000600190005000000B2
:10011000E000E300E200C35C01512C004C002A0027
:1001200027002600250024002300000031001300D2
:1001300012000C0018001C000000340033000F00F7
:100140000E000D000B0000002800380037003600BC
:100150001000110000004E004B002E002D00015138
:100160002C0028003A003B003C003D003E003F00D0
:1001700000000100C85CCA5CC95C005C2F00000084
:100180000100C75CCB5CC65C010001000000E1001F
:10019000010001000100010001000000E000E30097
:1001A000E200C45C0100010001004500440043007E
:1001B00042004100400000004A0049004E00520049
:1001C0004B00300000004D004C004F00510050002B
:1001D00001000000AB00AC00AE0001000100145CA7
:1001E0000000AA00A900A800010001000100010010
:1001F00000047F3F1F643214643214783C1E1E14C6
:100200000A052223252628292A2C2D2F3032333582
:1002100036383A3B3D3E4042434547494A4C4E50B2
:1002200051535557595A5C5E6062646668696B6DDC
:100230006F71737577797B7D7F81838587898A8CE0
:100240008E90929496989A9C9E9FA1A3A5A7A8AAE7
:10025000ACAEAFB1B3B4B6B8B9BBBCBEBFC1C2C31C
:10026000C5C6C7C9CACBCCCDCED0D1D2D2D3D4D5B6
:10027000D6D7D7D8D9D9DADADBDBDBDCDCDCDCDCDF
:10028000DDDDDDDDDCDCDCDCDCDBDBDBDADAD9D9B7
:10029000D8D7D7D6D5D4D3D2D2D1D0CECDCCCBCA45
:1002A000C9C7C6C5C3C2C1BFBEBCBBB9B8B6B4B36B
:1002B000B1AFAEACAAA8A7A5A3A19F9E9C9A989601
:1002C0009492908E8C8A89878583817F7D7B7977D4
:1002D0007573716F6D6B6968666462605E5C5A59B4
:1002E00057555351504E4C4A4947454342403E3D75
:1002F0003B3A3836353332302F2D2C2A2928262503
:100300002322FFAA7F5540000101010101010101E3
:1003100001020202020202020202030303030303B8
:100320000303040404040404040505050505060686
:100330000606060707070707080808080909090944
:100340000A0A0A0B0B0B0C0C0C0D0D0D0E0E0E0FEA
:100350000F0F10101111111212131314141515167A
:10036000161717181819191A1A1B1B1C1D1D1E1EEB
:100370001F2020212222232424252626272829293C
:100380002A2B2C2D2D2E2F30313232333435363767
:1003900038393A3B3C3D3E3F404142434445464765
:1003A00048494A4C4D4E4F50515354555658595A3E
:1003B0005B5D5E5F616264656668696B6C6D6F70E2
:1003C00072737577787A7B7D7E8082838587888A51
:1003D0008C8E8F91939596989A9C9EA0A2A3A5A788
:1003E000A9ABADAFB1B3B5B7BABCBEC0C2C4C6C984
:1003F000CBCDCFD1D4D6D8DBDDDFE2E4E7E9EBEE3D
:10040000F0F3F5F8FAFDFF1803500072006F006A70
:100410000065006300740020005A0065006E000053
:100420000010034C00650067006F006E00750074DB
:100430000000000403090409023B00020100A0FAC5
:10044000090400000103010100092111010001223A
:1004500040000705810308000109040100010300B1
:100460000000092111010001227B00070582032001
:1004700000011201000200000008EDFE60300100E2
:100480000102000105010902A10185020901A10083
:100490000509190129081500250195087501810232
:1004A0000501093009311581257F950275088106FE
:1004B00009381581257F950175088106050C0A38D4
:1004C000021581257F950175088106C0C0050109C7
:1004D00080A101850319012AB700150126B70095EF
:1004E0000175108100C0050C0901A10185041901E5
:1004F0002AA002150126A002950175108100C005F1
:10050000010906A101050719E029E7150025019554
:1005100008750181029501750881010507190029F7
:10052000FF150026FF0095067508810005081901D2
:100530002905950575019102950175039101C0008A
:1005400011241FBECFEFDAE0DEBFCDBF11E0A0E087
:10055000B1E0E2E0FEE502C005900D92AA3DB107D0
:10056000D9F723E0AAEDB1E001C01D92AE32B20787
:10057000E1F70E9427160C94FF2E0C940000CF93F5
:10058000DF93EC010E94350EBE0180E090E0DF9128
:10059000CF910C944408873A9D4551F4FB01828128
:1005A000882339F081E090E00E94BF0280E0089546
:1005B00081E0089581E008950C94CB0208950C9495
:1005C000DE021F93CF93DF9300D000D01F92CDB7F0
:1005D000DEB749835A836B833091DD0189819A812B
:1005E000311114C0662359F0222349F00E94990961
:1005F000182F682F89819A810E94420903C00E94A6
:100600006D09182F69817A81812F04C00E94990990
:1006100069817A810F900F900F900F900F90DF916A
:10062000CF911F910C94C510FC01262F4081518160
:100630006281738184810C94E10281E00895CF93FB
:10064000DF93EC0160E00E941403BE01DF91CF91C3
:100650000C94DF020C943B120C94371208950E9404
:10066000EC070E942E032FEF84E39CE02150804092
:100670009040E1F700C000000C9424270F931F93D3
:10068000CF93DF938C0161E00E941403EC01B80169
:100690000E94DC02882309F444C0B801CE010E9404
:1006A0005D238823F1F1B801CE010E94FA1F88234F
:1006B000C1F1B801CE010E94B922882391F1B8019D
:1006C000CE010E94E81E882361F1F801828188230F
:1006D00009F1CB358DE5D807C1F050F4C115FCE523
:1006E000DF0781F0CF3DDC45A9F40E94CF0E19C091
:1006F000CC35EDE5DE0761F0CD35DD4559F40E94DE
:10070000130E08C00E942F030CC00E941C0E02C0D2
:100710000E941F0EC801DF91CF911F910F910C9481
:10072000DA0280E0DF91CF911F910F9108950E942E
:100730003D260C94B0030E94B3030C944326089505
:100740000C949F0381E008950C94A2030895CF9325
:10075000C82F0E94A0038C2F0E94A403CF9108955C
:1007600080E00C94A7030E947B250C94A7030E94B1
:100770007B259091DC01891721F08093DC010C949A
:10078000A7030895CF93DF93CDB7DEB72B970FB6AE
:10079000F894DEBF0FBECDBF4F83588769877A8735
:1007A0008B8761110E945F0D9E012F5F3F4F86E096
:1007B000F90111928A95E9F785E0FE013796D90192
:1007C00001900D928A95E1F789819A814C815D8132
:1007D000452B31F09F3F31F491E08F3F19F403C076
:1007E00091E001C090E090FF09C049815A816B817E
:1007F0007C818D819E810E94800C05C0C9010E9470
:100800001D038111F2CF2B960FB6F894DEBF0FBEF9
:10081000CDBFDF91CF910895FC01808191810E942D
:10082000DB090895CF93882309F4A9C0C82F823823
:10083000C1F40E947B2581FDA2C069E38091020181
:10084000909103010E9415260E94810D2FEF81EEE9
:1008500094E0215080409040E1F700C0000069E33F
:1008600019C0833801F50E947B2580FD88C063E5AF
:1008700080910201909103010E9415260E94810D32
:100880002FEF81EE94E0215080409040E1F700C0CE
:10089000000063E580910201909103010E941726F8
:1008A000CF910C94810D8438C1F40E947B2582FD88
:1008B00066C067E480910201909103010E941526B1
:1008C0000E94810D2FEF81EE94E0215080409040F6
:1008D000E1F700C0000067E4DDCF8CEF8C0F813AB8
:1008E000F8F48C2F0E947022811149C06C2F8091E6
:1008F0000201909103010E94DF25882349F06C2FAB
:1009000080910201909103010E9417260E94810D9F
:100910006C2F80910201909103010E941526C0CF97
:1009200080E28C0F883048F4C77081E001C0880FE6
:10093000CA95EAF70E94420DB3CFEBE5EC0FE33026
:1009400040F4F0E0ED58FE4F808190E0CF910C94A0
:10095000A725E8E5EC0FE73150F4F0E0EE0FFF1FBC
:10096000EB5BFE4F80819181CF910C94BD25CD3EF4
:1009700030F08C2F0E94AC16CF910C947E17CF9143
:100980000895882309F464C0823879F40E947B2595
:1009900081FF5EC069E380910201909103010E9492
:1009A00015260E94810D69E310C08338B1F40E94BE
:1009B0007B2580FF4DC063E580910201909103018A
:1009C0000E9415260E94810D63E58091020190919D
:1009D00003010E9417260C94810D843879F40E943B
:1009E0007B2582FF35C067E480910201909103016D
:1009F0000E9415260E94810D67E4E7CF9CEF980FB7
:100A0000913A10F4682FE1CF90E2980F983050F4AB
:100A1000877091E001C0990F8A95EAF7892F0E94AB
:100A2000480DD9CF9BE5980F933020F480E090E0FB
:100A30000C94A72598E5980F973120F480E090E07A
:100A40000C94BD258D3E20F00E9407170C947E1754
:100A500008951F93CF93DF93182FEB010E94120488
:100A6000209741F08FE99FE00197F1F700C0000067
:100A70002197F6CF812FDF91CF911F910C94C10464
:100A8000893319F060E070E002C060E570E00C941A
:100A90002905882321F00E94420D0C94810D0895B0
:100AA000882321F00E94480D0C94810D0895CF9267
:100AB000DF92EF92FF920F931F93CF93DF937C010E
:100AC000D62FC72FFC011281058102950F700E945D
:100AD000380D8823B9F01123A9F08C2F807F803442
:100AE00021F080E28D0F883068F08091D10282FD84
:100AF00009C082E00E94E10D0E94380D91E0D82EDD
:100B0000D92601C0D12CCC2EC2948FE0C8228C2DC6
:100B100090E08C30910508F0CFC1FC01EA5AFF4FFC
:100B20000C945D2E8C2F807FCF70882311F0C2959E
:100B3000C07F112399F0CC2309F4AAC180E28D0F64
:100B4000883010F0D11104C08C2F0E94420D03C0D8
:100B50008C2F0E94520D0E94810D9AC18D2F0E94F0
:100B6000C104CC2309F4A8C180E28D0F883038F18C
:100B7000DD2329F18C2F0E94580D24C08C2F807FFB
:100B8000CF70803211F0C295C07FDD2319F0D130D3
:100B9000A1F13DC08091D10282FF17C0112349F01D
:100BA000CC2329F08C2F0E94420D0E94810D80E001
:100BB00070C180E00E94C104CC2309F47DC18C2F58
:100BC0000E94480D0E94810D77C1112371F000230E
:100BD00041F0013031F40E94620D8C2B0E946A0DAD
:100BE0006BC10E94620D8C2B1DC0002319F00130D7
:100BF00009F462C10E94770D25C0112321F006304F
:100C000008F05AC10EC0053008F056C11BC01123B0
:100C100061F0002331F0F701858180FF39C18F70C9
:100C200085838C2F0E94490547C1002359F0D93391
:100C300009F03FC1FFEF07EE13E0F1500040104014
:100C4000E1F735C18C2F0E94500536C18C2F869557
:100C50008695837019F0813061F02EC1112321F047
:100C60008D2F9C2F937002C080E090E00E94A725FA
:100C70002BC1112321F08D2F9C2F937002C080E097
:100C800090E00E94BD2520C18D2F112319F00E94F4
:100C9000AC1602C00E9407170E947E1715C18C2F48
:100CA000837009F047C011110BC12D2F2295269595
:100CB0002770220F220F6D2F6F70862F90E0A0E01B
:100CC000B0E0022E04C0880F991FAA1FBB1F0A9410
:100CD000D2F7D4FF10C04FE050E060E070E004C0F5
:100CE000440F551F661F771F2A95D2F740955095E0
:100CF0006095709503C040E050E0BA01C695C69576
:100D0000C3708A019B01082B192B2A2B3B2BC9018D
:100D1000B801C23049F058F4C13019F00E945808A7
:100D2000CFC00E944608CCC00E946A08C9C00E9479
:100D30004408C6C0112319F08C2F817001C086951C
:100D4000882309F4BDC02D2F229526952770220FE8
:100D5000220F6D2F6F70862F90E0A0E0B0E0022E82
:100D600004C0880F991FAA1FBB1F0A94D2F7D4FF93
:100D700010C04FE050E060E070E004C0440F551F29
:100D8000661F771F2A95D2F740955095609570950C
:100D900003C040E050E0BA01C695C695C3708A0111
:100DA0009B01082B192B2A2B3B2BC901B801C23000
:100DB00049F058F4C13019F00E941D0981C00E9409
:100DC0000B097EC00E942F097BC00E947E0878C05C
:100DD000CF70112339F08C2F0E94A4088D2F0E9410
:100DE00049056EC08D2F0E9450058C2F0E94C508AA
:100DF00067C0D23F21F128F4D03F41F0D13FC1F08C
:100E000043C0D33F19F1D43F79F03EC0112341F0E4
:100E1000053008F051C08C2F8F710E94EA084CC039
:100E2000063008F049C0F7CF8091D10282FF18C088
:100E3000112339F08C2F8F710E94A4083DC011231B
:100E4000C9F38C2F8F710E94C50836C0112329F079
:100E50008C2F8F710E948F082FC00E948A082CC08F
:100E6000112349F0CF718C2F0E94A40863E08C2FCE
:100E70000E94C60D21C081E00E94E10D0230E0F029
:100E800082E00E94E10D18C0112331F0002391F29D
:100E90008D2F0E94120410C0002399F2D93349F417
:100EA0001FEF27EE33E0115020403040E1F700C043
:100EB00000008D2F0E94C10488EF8C0D843020F437
:100EC0000E947B250E94A703DD20C9F00E94340DFB
:100ED00080FD15C0F70112820E942E0D0E94A40809
:100EE000C7010E94A0070E942E0DDF91CF911F9194
:100EF0000F91FF90EF90DF90CF900C94C508DF9199
:100F0000CF911F910F91FF90EF90DF90CF900895B8
:100F10000F931F93CF93DF93EC01688179818A81CE
:100F20000E94E6098C010E9441090E943208B80122
:100F3000CE010E945705DF91CF911F910F91089527
:100F4000CF93DF93EC01988189812B813C81232B06
:100F500031F08F3F31F481E09F3F19F403C081E00D
:100F600001C080E080FD1DC0CE010E943E038111C2
:100F700010C00E94380D8823A1F08A81882389F04F
:100F80008091D10282FD0DC082E0DF91CF910C945F
:100F9000E10DCE010E948807CE01DF91CF910C9424
:100FA0001F03DF91CF91089580E090E00E94A72574
:100FB00080E090E00E94BD250E945F0D0E94810D9F
:100FC0000E94AF180C947E1780910201909103014A
:100FD0000E9419260C94D4070E944F0D0C94E4072C
:100FE00092959F70963079F010F4925001C09A500B
:100FF000923068F4803F69F018F4883E40F409C0EC
:10100000843F29F406C0883E20F0813F11F080E043
:10101000089581E00895FC01808191810E94DB099F
:101020000E94F0070895CF93DF9300D000D01F9265
:10103000CDB7DEB70F900F900F900F900F90DF910C
:10104000CF910895CF93DF9300D000D000D0CDB7DB
:10105000DEB726960FB6F894DEBF0FBECDBFDF9188
:10106000CF910895089508950C9433080C94340892
:101070000E94360860930F02709310028093110251
:10108000909312020C94D4070C9438080F931F937A
:1010900000910F0210911002209111023091120262
:1010A000602B712B822B932B1F910F910C9438087E
:1010B0000F931F9300910F021091100220911102C3
:1010C0003091120260237123822393231F910F9189
:1010D0000C9438080F931F9300910F021091100287
:1010E00020911102309112026027712782279327E5
:1010F0001F910F910C9438080C9433080E947C08BF
:1011000060930B0270930C0280930D0290930E0279
:101110000C94D40760E070E0CB010C947E080F9330
:101120001F9341E050E060E070E08A019B0104C041
:10113000000F111F221F331F8A95D2F7C901B80172
:101140001F910F910C947E080F931F9341E050E084
:1011500060E070E004C0440F551F661F771F8A953A
:10116000D2F780910B0290910C02A0910D02B091E8
:101170000E028A019B01082B192B2A2B3B2BC9013C
:10118000B8011F910F910C947E080F931F9341E0BB
:1011900050E060E070E004C0440F551F661F771FE9
:1011A0008A95D2F7409550956095709580910B0285
:1011B00090910C02A0910D02B0910E028A019B0148
:1011C000082319232A233B23C901B8011F910F913A
:1011D0000C947E080F931F9341E050E060E070E0B4
:1011E00004C0440F551F661F771F8A95D2F7809160
:1011F0000B0290910C02A0910D02B0910E028A0197
:101200009B01082719272A273B27C901B8011F91ED
:101210000F910C947E080F931F9300910B02109175
:101220000C0220910D0230910E02602B712B822B4B
:10123000932B1F910F910C947E080F931F93009195
:101240000B0210910C0220910D0230910E026023CE
:101250007123822393231F910F910C947E080F9387
:101260001F9300910B0210910C0220910D023091FE
:101270000E0260277127822793271F910F910C94EC
:101280007E08089527E0929F800D1124E82FE695AF
:10129000E695E695877051E001C0550F8A95EAF70B
:1012A00085E0E89FF0011124E252FE4F20E030E09B
:1012B00070E04081CB01022E02C0969587950A947A
:1012C000E2F78170819584278523842781932F5F9E
:1012D0003F4F2530310569F7089527E0929F800D33
:1012E0001124682F669566956695982F977085E00E
:1012F000689FB001112440E050E080E0FB01E40F62
:10130000F51FE252FE4F208130E0092E02C03695D3
:1013100027950A94E2F721703327042E01C0220F8B
:101320000A94EAF7822B4F5F5F4F4530510531F742
:101330000895BF92CF92DF92EF92FF920F931F9387
:10134000CF93DF938C01C0900B02D0900C02E09001
:101350000D02F0900E0280910F0290911002A09168
:101360001102B0911202C82AD92AEA2AFB2ACFE137
:10137000D0E0D701C6010C2E04C0B695A79597956D
:1013800087950A94D2F780FD04C0219790F7B12C7D
:1013900007C0BC2EB8018C2F0E94D8100197A9F36A
:1013A0008B2DDF91CF911F910F91FF90EF90DF90E8
:1013B000CF90BF900895CF93DF93EC010E949909DD
:1013C000BE010E94D810DF91CF9108951F93CF9353
:1013D000DF93EB019091DD01992321F0CB010E9475
:1013E000DB0913C0882349F0CB010E949909182F0B
:1013F000682FCE010E94420904C0CB010E946D09F2
:10140000182FBE01812F0E94D810DF91CF911F911C
:1014100008951F93CF93DF93C091130216E080913C
:101420001402C81799F0D0E01C9FF0011D9FF00D29
:101430001124EB5EFD4F4081518162817381848173
:1014400095810E9422082196C770E9CFDF91CF9144
:101450001F910895409145025091460260914702C4
:10146000709148028091490290914A020C9422089E
:10147000EF92FF920F931F93CF93DF9380914A02D5
:1014800082958F7009F065C080914702882309F426
:1014900060C080911302F0901402109145020091F7
:1014A0004602609148027091490291E01F3F09F0A5
:1014B00090E0C0910001D0910101292F96E0E92E22
:1014C0008F1509F446C06115710521F00F3F21F019
:1014D00030E003C031E001C0322F90E030FD36C073
:1014E000E89EF001E99EF00D1124DF01AB5EBD4FD7
:1014F00011963C911197301329C03C91311326C0AD
:1015000012963C911297311121C013964D915C9126
:101510001497461B570B4C175D07C0F480914A0285
:101520008F70806180934A02E65EFD4F80818F70EC
:101530008061808385E492E00E94A007DF91CF91D3
:101540001F910F91FF90EF900C94090A01968770FC
:10155000B7CFDF91CF911F910F91FF90EF9008953A
:101560009F92AF92BF92CF92DF92EF92FF920F9332
:101570001F93CF93DF93CDB7DEB761970FB6F89483
:10158000DEBF0FBECDBF8C0185E0F801DE011D96E8
:1015900001900D928A95E1F7D8011296EC90909106
:1015A0004502E091460220914802309149022115FE
:1015B000310531F0EF3F31F481E09F3F19F403C072
:1015C00081E001C080E0B82FB1709B2E80FD47C143
:1015D000D8014C9111965C9111971396AD90BC90E7
:1015E000149785E4C82E82E0D82EF0904702B5010A
:1015F000621B730B2091000130910101FF2009F45F
:10160000D9C080914A026217730708F095C0282F4D
:10161000207F09F052C05E1313C0491311C0FE2C85
:10162000E1100EC08F70806180934A020E942A0AE6
:10163000C6010E94A00780914A02F80185834DC12E
:10164000AB2831F05F3F31F481E04F3F19F403C024
:1016500081E001C080E080FD03C081E08E2502C0F2
:1016600080E090E0F82FF170FF2E80FF1CC0809189
:1016700013022091140236E0821709F40BC190E0A6
:10168000389FF001399FF00D1124EB5EFD4F618111
:10169000561306C06081461303C06281E61203C080
:1016A00001968770E9CFFE2CEE2009F416C18091D7
:1016B0004A02816080934A0254C05E1306C04913F7
:1016C00004C0E11002C0F80199C0C8010E940B08D3
:1016D000882361F1EE2051F120914A02822F8295F8
:1016E0008F7090E0029774F08091450290914602CD
:1016F00098878F831986BB86AA862C87CE0107968A
:101700000E94A00786E0F801A5E4B2E001900D92E6
:101710008A95E1F70E94380A0E942A0A0AC05E17D9
:1017200011F1C8010E940B0881112CC0C8010E9450
:10173000A007FF24F394D1C0282F207F81F77A2DB2
:10174000B98AA88A6E2D89890E94130885E492E0DF
:101750000E94A00786E0D6011D928A95E9F70E94B3
:101760002A0AF12CBAC04913DCCFE110DACFF80114
:101770008583C8010E94A00786E0D6011D928A9544
:10178000E9F7ABC0EE2091F220914A02822F8295B8
:101790008F7090E002970CF4B5CF80914502909144
:1017A00046029A8389831B82BD82AC822E83CE013E
:1017B0000196A6CF6217730708F044C0FE2CEE20F6
:1017C00009F4B4CF5E1330C049132EC020914A02F1
:1017D00020FD21C0822F82958F70482F50E0411547
:1017E0005105C9F0F80125834F30510541F08F5F55
:1017F000982F9295907F822F8F70892B8583C801B7
:101800000E94A00786E0F801A5E4B2E001900D92E5
:101810008A95E1F73CC086E0F801A5E4B2E00190CA
:101820000D928A95E1F759C0C8010E940B088111F9
:1018300069CF80914A02816080934A02C8010E9468
:10184000A0074BC07A2DB98AA88A6E2D89890E947B
:10185000130886E0D6011D928A95E9F718C0EE209C
:1018600009F464CFC8010E940B08F82E882309F4FC
:101870005DCF86E0F801A5E4B2E001900D928A9573
:10188000E1F785E492E00E940C040E94380A0E946D
:101890002A0A23C04D875E878D859E850E94DB09BD
:1018A000292F22952F70223028F49F7039F0811152
:1018B00005C00BC0243028F49F7049F4805E883046
:1018C00020F0C8010E94A0079F2CF92C06C0D80167
:1018D00015969C91907F91F7F8CF8F2D61960FB65A
:1018E000F894DEBF0FBECDBFDF91CF911F910F9156
:1018F000FF90EF90DF90CF90BF90AF909F900895B2
:101900001F93CF93DF93CDB7DEB72C970FB6F89424
:10191000DEBF0FBECDBF4F83588769877A878B871D
:101920009C87CE0107960E94B00A8823D1F09F8140
:1019300088852A853B85232B31F08F3F31F481E068
:101940009F3F19F403C081E001C080E080FD47C0E3
:101950004F81588569857A858B859C850E942208F0
:101960003EC086E0FE013796DE01119601900D9291
:101970008A95E1F7FF81E8856A857B8561157105A8
:1019800031F0EF3F31F481E0FF3F19F403C081E013
:1019900001C080E080FD23C02091140230E0C90125
:1019A0000196877099274091130250E0841795079C
:1019B000F1F1F983EA837D836C8396E0929FD001F5
:1019C000939FB00D1124AB5EBD4FFE013196019087
:1019D0000D929A95E1F7809314020E94090A16E08D
:1019E0008091130290911402891771F1189FC00120
:1019F00011248B5E9D4F0E94B00A882329F1E0914B
:101A000013021E9FF0011124EB5EFD4F40815181B6
:101A100062817381848195810E94220880911302E2
:101A200090E001968770992780931302D9CF0E9486
:101A3000EC071092140210921302E5E4F2E086E043
:101A4000DF011D928A95E9F72C960FB6F894DEBF58
:101A50000FBECDBFDF91CF911F91089580915302AA
:101A60008595859585950895809153028770089591
:101A700090915302977081E009F480E0089580917D
:101A80005E02089590915E02892B80935E02089514
:101A9000809590915E02892380935E020895109252
:101AA0005E02089590915D02892B80935D020895F6
:101AB000809590915D02892380935D020895109234
:101AC0005D02089580915402089508950C94650D67
:101AD0000C94660D9091D10292FD08C09091540231
:101AE000981721F0809354020C94680D089580910A
:101AF0005402882329F01092540280E00C94680D5F
:101B00000895CF93DF93E0910201F091030180915A
:101B10005E028083E0910201F09103019081809147
:101B20005D02892B808380915402882381F0E091AB
:101B30000201F09103019081892B80838091020141
:101B4000909103010E94D32581110E94770DC091CD
:101B50000201D091030148E050E06BE472E0CE0155
:101B60000E94A12E892B69F088E0FE01ABE4B2E06F
:101B700001900D928A95E1F7CE01DF91CF910C94FF
:101B80008E25DF91CF9108950C94650D9091D1022F
:101B900092FD10C098E0899F90011124262B20937C
:101BA00053020E94A40880915302859585958595DE
:101BB0000C94C40D0C94A4081092530280E00C9471
:101BC000C40D209153028095822380935302982F55
:101BD000977099F430E0482F082E000C550B24170D
:101BE000350759F09091D10292FD07C085958595F2
:101BF00085950E94C5080C94DC0D08959091D10242
:101C000092FB222720F9281769F080FB92F9909324
:101C1000D1028091D0029091D1020E944B0E82E0BD
:101C20000C94E10D08958091D10282FB882780F900
:101C300091E089270C94FE0D81E00C94FE0D80E06C
:101C40000C94FE0D80E090E00E94C52E21E0893EBC
:101C50009E4F09F020E0822F089582E090E00C94DE
:101C6000B72E83E090E00C94B72E682F83E090E0CD
:101C70000C94CB2ECF9384E090E00E94B72EC82F17
:101C800082E290E00E94B72E2C2F30E0A901582B61
:101C9000CA01CF910895CF93C92F682F84E090E0B7
:101CA0000E94CB2E6C2F82E290E0CF910C94CB2E31
:101CB000AB01BC018FE090E00C94DD2EAB01BC01C8
:101CC00083E190E00C94DD2E60E070E0CB010C9499
:101CD0005E0E60E070E0CB010E94580E0C94640E22
:101CE00069EE7EEF80E090E00E94E92E60E082E005
:101CF00090E00E94CB2E60E083E090E00E94CB2E2B
:101D000010920F0210921002109211021092120201
:101D100060E084E090E00E94CB2E60E082E290E000
:101D20000E94CB2E60E085E090E00E94CB2E60E028
:101D300086E090E00E94CB2E6FEF87E090E00E945B
:101D4000CB2E40E050E0BA0188E090E00E94DD2E0A
:101D500060E08DE090E00E94CB2E40E050E0BA01C0
:101D600088E190E00E94DD2E60E087E190E00E9433
:101D7000CB2E40E050E0BA018CE190E00E94DD2ED5
:101D800060E070E080E290E00E94E92E40E050E0E8
:101D9000BA0188E190E00E94DD2E0C94690E0C944B
:101DA000700E682F8EE090E00C94CB2E0E94C72618
:101DB00060936D0270936E0280936F029093700235
:101DC0006093690270936A0280936B0290936C0235
:101DD000089585B7806885BF85B7806885BF0895F9
:101DE0000C94EF1308950C94F20E0C94F20E0C94D4
:101DF000F50E0C94F20E0C94F90E0C94F20E0E9457
:101E0000E90E8EEF91E10E9471250E94FD0E0C9467
:101E1000FB0E0E94F30E0C94F20E0E9401120C9421
:101E2000A6030E94B2260E94B4110E9409140E94C7
:101E300040130E940D0F0E94E21F0E94071E0E9485
:101E400013140C94F70E8F929F92AF92BF92CF9281
:101E5000DF92EF92FF920F931F93CF93DF93CDB753
:101E6000DEB72A970FB6F894DEBF0FBECDBF0E9433
:101E70006413982E81110E94D60E8FE5A82E82E061
:101E8000B82E00E010E0802E802F0E942512D82E60
:101E9000F501C1905F01C826B1F40F5F1F4F0A30F2
:101EA000110589F78FEF89838A831B820E94BB26E5
:101EB0008160782F9D838C8349815A816B818D81CC
:101EC0000E94C2032FC08091710281FD0E942B12DB
:101ED000E12CFF24F3948C2D8F21F1F00E94F00E61
:101EE000882399F0EE828F82DF2081E009F480E080
:101EF00088870E94BB268160782F9A8789874E81C8
:101F00005F8168858A850E94C203F801E15AFD4F0E
:101F10008081F826F08206C0E394FF0CF7E0EF1210
:101F2000DACFBBCF81E0911001C080E02A960FB6D6
:101F3000F894DEBF0FBECDBFDF91CF911F910F91FF
:101F4000FF90EF90DF90CF90BF90AF909F908F90D9
:101F500008950E94230F0E94EF130E943A1E0E94D0
:101F60009C170C94B703CF93DF930E94DD10EC0114
:101F7000811521E5920708F045C0811530E59307EA
:101F800008F094C0883E910528F5803E910508F040
:101F9000F8C0883A910570F4853A910508F07CC044
:101FA0008130910509F475C008F4E8C0049708F081
:101FB000E8C0E4C08F3B910508F0E0C0C85AD0E00B
:101FC000CC0FDD1FCA58DE4F0990D881C02DCE013D
:101FD0009464D8C0811540E2940758F4811551E00B
:101FE000950708F0CEC08D3E910508F4C7C09065F6
:101FF000C9C0C11580E4D80708F4C0C0DF70CE01A5
:10200000906AC0C0811525E59207A8F4811534E5D2
:10201000930708F095C0811543E5940708F07BC04D
:10202000811552E5950708F061C0D82FCC27CE0165
:10203000816F906AA7C0C11589E5D807A0F4C115C2
:1020400028E5D20708F082C0C11536E5D30708F0AD
:1020500095C08C2F0E9471118F7190E0D82FCC27E2
:10206000CE0190628FC0C1154AE5D40708F474C050
:10207000CE0190568115904208F080C08D2F8F714F
:102080000E947111DD27D0628F71AE01582BCA01F9
:1020900079C081E090E076C0C55AD0E0CC55DE4FE3
:1020A0008881C82FD0E0CE0190646CC074E0969512
:1020B00087957A95E1F7282F23703C2F337081E0C4
:1020C00090E002C0880F991F3A95E2F79C68AC0136
:1020D000522B9A019C2F9F709695969550E2959F52
:1020E000E0011124C9018C2B9D2B4CC083709927D2
:1020F00021E030E002C0220F331F8A95E2F79C2FC7
:102100009695969580E2989FE0011124C22BD32BDF
:10211000CE019C6837C08370992721E030E002C06F
:10212000220F331F8A95E2F79C2F9695969540E2F1
:10213000949FE0011124C22BD32BCE019A6822C0B8
:10214000D82FCC27CE01846F906A1CC0DC2FCC27FF
:10215000CE01806F906A16C08C2F8F700E94711113
:1021600094E0D695C7959A95E1F7CF70D0E0DC2F33
:10217000CC27D0699E01282BC90104C080E090E0E3
:1021800001C0CE01DF91CF91089526E4829FC00166
:102190001124FC0127E0729FE00DF11D1124E60FD0
:1021A000F11DEE0FFF1FE852FF4F859194910895A6
:1021B0000E94C5100E94B30F08958238910569F1FD
:1021C000B0F48133910509F46DC048F4893291056A
:1021D00009F463C08A32910509F469C00895853312
:1021E000910509F455C089339105B9F00895833EEE
:1021F000910569F138F4803E9105B1F0823E910578
:1022000009F10895863E9105A9F1873E9105B9F13E
:10221000843E910509F064C023C02091D00220FDC6
:102220004FC021FD4DC008958091D00280FD44C073
:102230008091D10280FF44C08091D00284FD42C0D1
:1022400083EE4DC08091D00282FF38C0F5CF8091DF
:10225000D00282FD33C08091D10280FD31C0ECCF2D
:102260008091D10281FF32C08091D00284FD2AC0CA
:1022700087EE35C08091D00283FF26C0F5CF8091D4
:10228000D00283FD21C08091D10281FD1FC0ECCF1F
:102290008091D00285FD1CC01DC08091D00285FDBB
:1022A00019C016C08091D00286FD16C017C080915B
:1022B000D00286FD13C010C089E311C082EE0FC0AA
:1022C00080EE0DC080E00BC086EE09C084EE07C032
:1022D00089E205C085E303C08AE201C081E390E0A2
:1022E00008959091D00292FF0DC0282F28712830B8
:1022F00019F4877F846006C0282F2471243011F4DC
:102300008B7F886093FF0DC0282F2871283119F426
:10231000877E846106C0282F2471243111F48B7EBE
:1023200088612091D10220FF0DC0382F38713830DC
:1023300019F4877F816006C0382F3171313011F474
:102340008E7F886021FF0DC0282F2871283119F455
:10235000877E816106C0282F2171213111F48E7E84
:10236000886194FD877E08951092CC021092CD0270
:102370001092CE021092CF020895CF92DF92EF9288
:10238000FF926B017C010E94EF1381110EC00E942D
:10239000C726C61AD70AE80AF90AC092CC02D09218
:1023A000CD02E092CE02F092CF02FF90EF90DF904C
:1023B000CF9008950F931F930E94EF13882321F06D
:1023C0001F910F910C94C7260E94C7260091CC0242
:1023D0001091CD022091CE023091CF02600F711F7B
:1023E000821F931F1F910F9108950E94EF13811177
:1023F0000C94BB260E94DA11CB01089580E0089569
:1024000008950E94220E811102C00E94CF0E0E94E8
:102410002D0E809371020E943A0E9093D102809308
:10242000D0020E9400120E94310E682F70E080E0FE
:1024300090E00E94440860910B0270910C02809120
:102440000D0290910E020C947C08E82FF0E0E3520C
:10245000FD4F80810895089580EA8A95F1F70895E7
:1024600000C008950C942C1208950C9434120C940E
:1024700035120C9434120C9439120C943412FF92CD
:102480000F931F93CF93DF9300D000D01F92CDB74F
:10249000DEB70E94EF136091E7028823E9F185E03F
:1024A000F82E8E010F5F1F4FF8018F2D11928A9524
:1024B000E9F7862F90E0B80183529D4F0E942114C6
:1024C000882389F08091D20290E045E050E0B80185
:1024D00083529D4F0E94A12E21E020937202892BEE
:1024E00061F410E016C0809172028823D1F3F801E4
:1024F0001192FA94E9F710927202A091D202B0E020
:10250000A352BD4F85E0F80101900D928A95E1F745
:1025100011E00E942C030DC070E063527D4F80914A
:10252000D20290E083529D4F0E94AB140E943D1254
:1025300010E0812F0F900F900F900F900F90DF9170
:10254000CF911F910F91FF900895F894E82FE29595
:10255000EF70F0E031A1282F2F7081E090E001C0F2
:10256000880F2A95EAF7982F9095932391A392A12B
:10257000892B82A3789408950F931F93CF93DF93B1
:10258000CEEAD1E089918F3F11F00E94A51281E03F
:10259000C33BD807B9F7C7EAD1E00EEA11E0899149
:1025A0008F3F11F00E94A5120C171D07C1F7DF9194
:1025B000CF911F910F910895CF92DF92EF92FF92EA
:1025C0000F931F93CF93DF938C01C62FD0E0CE01E2
:1025D00082559E4F7C01FC0190819F3F09F447C0CA
:1025E000D62EF894E92FE295EF70F0E081A19F706C
:1025F00021E030E001C0220F9A95EAF7822B81A3F7
:1026000082A12095282322A378940E943012E7EA21
:10261000F1E04EEA51E031E0C12C21912F3F89F0E9
:10262000A22FA295AF70B0E090968C9190E02F70A1
:1026300002C0959587952A95E2F780FD02C0832F09
:1026400001C080E0C82A330F4E175F0731F7F7014A
:1026500080818F3F11F00E94A51261E0C11001C07E
:1026600060E08D2D0E943212C00FD11FC882DF9111
:10267000CF911F910F91FF90EF90DF90CF90089531
:102680008091040180910401811102C095E001C094
:1026900090E09093E70285E0891B8093D2020E942C
:1026A000BC128AE0EDEDF2E0DF01982F1D929A95C1
:1026B000E9F7E3EDF2E0DF011D928A95E9F785E0A5
:1026C0000E94B8130C942A03EF92FF920F931F936A
:1026D000CF93DF93CDB7DEB72A970FB6F894DEBF5E
:1026E0000FBECDBF8E010F5F1F4F8AE0F801119220
:1026F0008A95E9F7F12C6F2DC8010E94DC12F39442
:10270000F5E0FF12F8CF4AE050E0B80183ED92E027
:102710000E94A12E7C0121E0892B09F420E0E11424
:10272000F10441F08AE0F801A3EDB2E001900D92CE
:102730008A95E1F76091E70270E063527D4F45E0D2
:1027400083ED92E00E94B913EF2819F40E943F1222
:1027500002C081E090E02A960FB6F894DEBF0FBE6B
:10276000CDBFDF91CF911F910F91FF90EF90089512
:102770000895FF920F931F93CF93DF938C01F62E52
:10278000D72FC42F222349F081E0809375020E9445
:10279000BB26909374028093730280917502882304
:1027A000C1F080917302909174020E94D326059724
:1027B00080F0EF2DFD2FD8014C2F50E0CD01801B74
:1027C000910B841795071CF48D918193F7CF10928C
:1027D0007502DF91CF911F910F91FF900895809125
:1027E000780281110DC00E94062E811102C082E084
:1027F00001C081E080937802823011F40E94012EA2
:1028000081E090917802913009F080E008950C9475
:10281000EF130E940714809304010E94EF138111AB
:102820000C94591408950E94EF13811102C00C9466
:102830005B14089581E0909179029A3008F080E06D
:1028400008950F931F93CF93DF93EC018B01809139
:1028500079028A3038F4B801CE010E94A91481119E
:102860001DC00AC080917602909177020E94D32603
:10287000843F914080F715C0809179028F3F19F015
:102880008F5F80937902809179028A3060F00E9494
:10289000BB26909377028093760203C01092790250
:1028A00002C080E001C081E0DF91CF911F910F91C4
:1028B00008950C940A240C940D24DF92EF92FF9259
:1028C0000F931F93CF93DF937901C82F880FDD0BF0
:1028D00041155105A9F0FE0193E0EE0FFF1F9A95F7
:1028E000E1F7EB5FFE4F8181928186589D4F2081F9
:1028F00030E04217530708F49A01A9010E94AE2E56
:10290000CE010E94F624D82E8823D1F0011511059E
:10291000B9F083E0CC0FDD1F8A95E1F7FE01EB5F94
:10292000FE4F438150E00417150708F4A801CB5F60
:10293000DE4F6C817D8166587D4FC7010E94AE2EAF
:102940008D2DDF91CF911F910F91FF90EF90DF9030
:1029500008950C94C5150C94E1150F931F93CF9314
:10296000DF9300D000D0CDB7DEB7609191027091B7
:10297000920280919302909194020E94E226643622
:1029800071058105910528F10E94DA11DC01CB0166
:102990000296A11DB11D89839A83AB83BC8300E09D
:1029A00010E020E030E044E050E0BE016F5F7F4F78
:1029B00082E00E945D14182F882361F00E94C726D0
:1029C0006093910270939202809393029093940289
:1029D00001C011E0812F0F900F900F900F90DF91A9
:1029E000CF911F910F910895AF92BF92CF92DF9236
:1029F000EF92FF920F931F93CF93DF937C015B01C4
:102A00006A010E941A14811103C001E010E002C0A3
:102A10000AE010E0C1E0D0E0F894B501C701F6018A
:102A200009957894811115C021960C171D0794F013
:102A3000CC9F9001CD9F300D300D112480E090E0AF
:102A400045E34A95F1F70000019682179307C1F715
:102A5000E3CF81E0DF91CF911F910F91FF90EF9035
:102A6000DF90CF90BF90AF900895AF92BF92CF927A
:102A7000DF92EF92FF920F931F93CF93DF9300D0DB
:102A800000D000D0CDB7DEB77B01C090B301D090AD
:102A9000B40101E010E09E012A5F3F4F40E050E0AA
:102AA00060E070E080E00E945D14182F882309F434
:102AB0003EC056018FEFA81AB80A60918D0270913E
:102AC0008E0280918F02909190020E94E2266436DD
:102AD00071058105910518F105E010E09E012F5F59
:102AE0003F4F40E050E060E070E081E00E945D1404
:102AF000182F65E070E0C5010E94E31F91E02E8170
:102B0000281390E0192339F10E94C72660938D02A3
:102B100070938E0280938F029093900211C065E0B3
:102B200070E0C5010E94E31F9E818913D5CF85E027
:102B3000F6013196DE01119601900D928A95E1F72A
:102B4000112349F085E0FE013196A8E8B2E001903A
:102B50000D928A95E1F785E0E8E8F2E0D70101906F
:102B60000D928A95E1F7812F26960FB6F894DEBF75
:102B70000FBECDBFDF91CF911F910F91FF90EF90CE
:102B8000DF90CF90BF90AF9008950F931F93CF9396
:102B9000DF93EC018B0145E355E10E94F414882397
:102BA00051F04DEA54E1B801CE01DF91CF911F9170
:102BB0000F910C94F41480E0DF91CF911F910F914D
:102BC00008950F931F93CF93DF93F894C091B301AF
:102BD000D091B401CE01019625E0FB01DC0101900A
:102BE0000D922A95E1F765E070E00E94E31F88836B
:102BF0007894F8946E817F8188859985009184020C
:102C0000109185022091860230918702601771072A
:102C10008207930751F0609384027093850280933A
:102C20008602909387020E94BD117894DF91CF9124
:102C30001F910F9108950E94C7280E94110F0C94B4
:102C4000D3280E94D7280E94A90F0C94F1280E9433
:102C500059260E94AE280E94FF0E0E941B160E9459
:102C600021160E94090FFBCF80919B0280FF06C0B6
:102C70006091220170E0660F771F26C081FF04C0BB
:102C80006091220184E005C082FF07C060912201AB
:102C900088E0689FB001112417C090919A0299238F
:102CA000D1F060912101961788F72091220188E0E8
:102CB000289F90011124929FA001939F500D1124F1
:102CC00070E0CA010E94272E6038710540F461153A
:102CD000710519F406C068E070E0862F08958FE74B
:102CE000089581E0089580919B0280FF08C0609163
:102CF0001E0170E0759567957595679521C081FFF8
:102D000006C060911E0170E07595679519C082FF3D
:102D100004C060911E0170E010C090919902992347
:102D200099F060911D019617A0F780911E01899F6F
:102D3000C001112470E00E94272E6038710540F414
:102D40006115710519F406C061E070E0862F0895E1
:102D50008FE7089581E008958D3E21F40E94341696
:102D6000819504C08E3E29F40E94341680939F0200
:102D700008958F3E21F40E943416819504C0803F4F
:102D800029F40E94341680939E020895893F19F415
:102D90000E94731605C08A3F31F40E947316819514
:102DA0008093A00208958B3F21F40E9473168195B1
:102DB00004C08C3F29F40E9473168093A1020895E9
:102DC0009FE0980F983078F421E030E0A90102C02C
:102DD000440F551F9A95E2F7CA0190919D02892BE5
:102DE00080939D0208958D3F21F480919B02816024
:102DF0000BC08E3F21F480919B02826005C08F3F03
:102E000029F480919B02846080939B0208958D3EFB
:102E100039F490919F0297FF35C010929F0259C0DC
:102E20008E3E29F490919F021916BCF32BC090910D
:102E30009E028F3E29F497FF25C010929E0249C042
:102E4000803F19F41916CCF31DC09091A002893F60
:102E500029F41916BCF41092A0023BC08A3F19F461
:102E600097FF10C0F8CF8B3F39F49091A10297FFE4
:102E700009C01092A1022DC08C3F21F49091A102B3
:102E80001916BCF39FE0980F983080F421E030E0F1
:102E9000A90102C0440F551F9A95E2F7CA01809517
:102EA00090919D02892380939D0213C08D3F21F450
:102EB00080919B028E7F0BC08E3F21F480919B02FC
:102EC0008D7F05C08F3F29F480919B028B7F80937B
:102ED0009B0280919E02811106C080919F02811108
:102EE00002C010929A028091A002811106C08091C6
:102EF000A102811102C01092990208950E94BB267E
:102F000020919E02211104C020919F02222321F0D2
:102F100090939802809397022091A002211104C0FF
:102F20002091A102222321F0909396028093950292
:102F30008CE992E00C949925EF92FF920F931F93E6
:102F4000CF93DF9300D000D000D0CDB7DEB786E0BE
:102F5000ECE9F2E0DE01119601900D928A95E1F71D
:102F6000E0909E02F0909F020091A0021091A102B9
:102F700010929E0210929F021092A0021092A10243
:102F8000E11003C0FF2009F45DC080919702909189
:102F900098020E94D326AC0190919A02992339F0AD
:102FA0002091230130E02417350758F04BC02091C1
:102FB00024018AE0289F900111242417350718F076
:102FC00041C09F3F19F09F5F90939A02EE2061F0FD
:102FD0000E9434161E1414F09FEF01C091E0989FD8
:102FE000902D112490939E02FF2061F00E943416D0
:102FF0001F1414F09FEF01C091E0989F902D1124B1
:1030000090939F0230919E023323E1F020919F0222
:103010002223C1F045EB3403C0011124992319F098
:1030200090939E0203C081E080939E0235EB2303C0
:10303000C0011124992319F090939F0203C081E0ED
:1030400080939F02011103C0112309F45DC0809198
:103050009502909196020E94D326AC01909199021C
:10306000992339F020911F0130E02417350758F0DB
:103070004BC0209120018AE0289F90011124241741
:10308000350718F041C09F3F19F09F5F9093990258
:10309000002361F00E947316101614F09FEF01C018
:1030A00091E0989F902D11249093A002112361F03C
:1030B0000E947316111614F09FEF01C091E0989FC3
:1030C000902D11249093A1023091A0023323E1F0BE
:1030D0002091A1022223C1F045EB3403C001112449
:1030E000992319F09093A00203C081E08093A0027D
:1030F00035EB2303C0011124992319F09093A10209
:1031000003C081E08093A10280919E0281110BC0D7
:1031100080919F02811107C08091A002811103C09C
:103120008091A10281110E947E17EB82FC820D83A7
:103130001E8386E0FE013196ACE9B2E001900D926B
:103140008A95E1F726960FB6F894DEBF0FBECDBF85
:10315000DF91CF911F910F91FF90EF900895ECE9CF
:10316000F2E086E0DF011D928A95E9F710929A025B
:103170001092990210929B020895EF92FF920F9382
:103180001F93CF93DF938B01682F11110AC0442343
:1031900029F0E82FF0E0E95FFC4F6491762F862F4D
:1031A00075C0212F30E0E82FF0E0442321F0E95FE3
:1031B000FC4FE491F0E046E0049FC0011124CFEF02
:1031C000D0E0BE010E94132E4BEA4603C001479F88
:1031D000900D1124800F911D800F911D982F990F34
:1031E000890FAE01421B530B4E9FD0014F9FB00D74
:1031F0005E9FB00D11249B2F189FA0011124452F15
:1032000055278E01041B150B0E9FA0010F9F500D1B
:103210001E9F500D11247E01E81AF108E29E8001E4
:10322000E39E100DF29E100D1124212F3327C21B97
:10323000D30BCE9F9001CF9F300DDE9F300D112418
:1032400062307105A9F048F46115710569F06130CB
:103250007105C9F48B2F752F0DC06430710581F095
:1032600058F06630710579F47E2F8B2F932F0DC0A7
:10327000832F7B2F9E2F09C08E2F7B2F952F05C06C
:103280008E2F732F02C07E2F852F692FDF91CF9154
:103290001F910F91FF90EF90089541E00E94BD189B
:1032A000089508950E944D190895CF93DF93762FC6
:1032B000E901682F842F0E945219798368838A83D9
:1032C000DF91CF9108958091E802282F269530E074
:1032D0002115310519F48170826005C02532310550
:1032E00024F0817088648093E802089588E090E07B
:1032F0000C94BF2ECF92DF92EF92FF926B017C0174
:103300000E946319B701A60188E090E0FF90EF905A
:10331000DF90CF900C94DD2EE8EEF2E083E0808326
:1033200011828FEF82838383148260817181828115
:1033300093810C947A198091E80280FF02C08695EF
:10334000089580E008959091EC02933018F49F5F07
:103350009093EC02882351F06091E8027091E902A9
:103360008091EA029091EB020C947A19089581E021
:103370000C94A3199091EC02992319F09150909319
:10338000EC02882351F06091E8027091E90280918B
:10339000EA029091EB020C947A19089581E00C9462
:1033A000BA1970E00C94B71F609129018091E8026E
:1033B00080FF0AC08091280123E0829FC001112470
:1033C00083519D4F0C94D11980912A0190912B012A
:1033D000891780F7E82FF0E09F01220F331FE20FDB
:1033E000F31FE351FD4F1182108212828F5FF0CFE5
:1033F0009091E80290FF16C090912A0120912B0134
:10340000921770F4E92FF0E0DF01AA0FBB1FEA0F5B
:10341000FB1FE351FD4F8183608342839F5FF0CFA9
:103420000C94D4190895CF93DF9300D01F92CDB799
:10343000DEB79091E80290FF0AC09E012F5F3F4FD8
:103440000E9455194B8169818A810E94F8190F9059
:103450000F900F90DF91CF910895CF93DF93EC0100
:10346000EC81F0E0EE5FFD4F4491E8EEF2E0628126
:1034700081810E94131A8C818F5F8C83DF91CF91A1
:103480000895CF93DF93EC01E8EEF2E0438162818F
:103490008C810E94131A8C818F5F8C83DF91CF9176
:1034A00008950F931F93CF93DF9300D01F92CDB752
:1034B000DEB78C018091A20281110AC09E012F5FAC
:1034C0003F4F4FEF6FEF0E9455198A818093A20200
:1034D000F8018481813051F028F0823061F440910C
:1034E000A2020AC08091A20240E007C06091A2023D
:1034F00040E080E003C040E080E060E00E94F81916
:10350000F801848190E0019663E070E00E94272E2C
:1035100084830F900F900F90DF91CF911F910F91A7
:103520000895AF92BF92CF92DF92EF92FF920F93E6
:103530001F93CF93DF9300D01F92CDB7DEB7182F24
:10354000F62E042FE22E9091E80290FF6DC0E92F35
:10355000E695AE2FB0E0AB54BE4F8C918093AC0299
:103560009E7F923061F49E012F5F3F4F812F0E941A
:1035700055194B8169818A810E94F81943C08230B4
:1035800019F40091EB023EC0863019F41091E90263
:1035900039C08930D9F38931A9F5E9518E2F81706D
:1035A000D82EE695F0E0EE5FFC4FA590B490C12CCC
:1035B000BB2460912C01C61618F52C2D30E0A29E7C
:1035C000C001A39E900DB29E900D112470E00E9448
:1035D000132E812FD11002C0860F01C0861B90913F
:1035E0002A01290F311DA901440F551F240F351F32
:1035F00023513D4F402F6F2D0E945519C394D9CFB1
:103600000E94D4191093E902F092EA020093EB02AF
:10361000EE2051F06091E8027091E9028091EA0297
:103620009091EB020E947A190F900F900F90DF910A
:10363000CF911F910F91FF90EF90DF90CF90BF90AF
:10364000AF900895E8EEF2E09181282F43816281E6
:1036500088E0890F0C94911A81E00C94221BE8EE0B
:10366000F2E09181282F4381628188EF890F0C94C9
:10367000911A81E00C942F1BE8EEF2E0628128E0C1
:10368000620F08F46FEF282F438181810C94911A07
:1036900081E00C943C1BE8EEF2E0628128E0621BC2
:1036A00008F460E0282F438181810C94911A81E015
:1036B0000C944B1BE8EEF2E0438128E0420F08F443
:1036C0004FEF282F628181810C94911A81E00C9434
:1036D0005A1BE8EEF2E0438128E0421B08F440E088
:1036E000282F628181810C94911A81E00C94691BCE
:1036F00020E00C94911AFF920F931F93CF93DF93C6
:10370000EC01F12C0FEF10E060912C01F616F0F4B3
:1037100080912A012F2D30E0280F311DC901880F1B
:10372000991F280F391F23513D4F70E0C8010E9497
:10373000272E962F8C814091EB026091EA02F99E30
:10374000800D11240E945519F394DECF0E94D419E4
:103750009A818C8190FF02C08F5F01C081508C8361
:10376000DF91CF911F910F91FF900895BF92CF925B
:10377000DF92EF92FF920F931F93CF93DF93FC01A1
:10378000828180FF02C00FEF01C001E010E0809154
:103790002C01181708F040C080912A01C12ED12CAD
:1037A000E601C80FD11DCE01880F991FC80FD91F80
:1037B000C351DD4F198218821A8234E0E32EF12CB6
:1037C000B12C8091A4028B0D813114F08F7005C053
:1037D00087FF03C090912C01890F082E000C990BD4
:1037E000C816D90691F48091EB028E9DA0018F9DA1
:1037F000500D112455954795559547959E0160911B
:10380000EA028091E9020E945519B00EF1E0EF1A28
:10381000F108B9F61F5FBBCF0E94D4198091A402B2
:10382000013031F4811102C080912C01815007C018
:1038300090E0019660912C0170E00E94272E809309
:10384000A402DF91CF911F910F91FF90EF90DF9035
:10385000CF90BF900895CF9380912A0190912B0132
:10386000891770F4E82FF0E09F01220F331FE20F59
:10387000F31FE351FD4F1182108212828F5FF0CF50
:10388000C0E060912C01C617C0F5EC2FF0E070E0AD
:10389000CF010E94272E20912A01820F2091A3029E
:1038A000022E000C330B90E0E217F307CCF02091CE
:1038B0002701022E000C330B2E173F078CF09C01C2
:1038C000220F331F820F931F9C0123513D4F4091C4
:1038D000EB026091EA028091E9020E9455190BC047
:1038E000FC01EE0FFF1F8E0F9F1FFC01E351FD4FE8
:1038F000118210821282CF5FC4CF0E94D41920910E
:1039000026018091A302820F8093A3029091270148
:10391000920F9093270119165CF4082E000C990B56
:1039200040912C0150E041505109841795071CF03B
:10393000219520932601CF9108958F929F92AF9267
:10394000BF92CF92DF92EF92FF920F931F93CF938C
:10395000DF938C01FC014481C42FD0E09E01DE0185
:103960000E946B2E9B01AC010E94812E6B017C0199
:10397000E0E2F0E0EC1BFD0BA5E5B0E09B01AC0143
:103980000E94812E4B015C019F01DF010E94632E8A
:103990009B01AC010E948C2E9B01AC012C0D3D1DA6
:1039A0004E1D5F1DC501B4010E943B2EC22FD22FB8
:1039B0002A3228F4F3E02F9F900111240DC025E551
:1039C00030E02C1B3109C901880F991F280F391FBE
:1039D00037FF02C02F5F3F4F35952795C22FC09507
:1039E000F12C85E5E82EED1A80912C01F816C8F42B
:1039F000F1FC02C08E2D01C08D2F90912A012F2D38
:103A000030E0290F311DA901440F551F240F351F28
:103A100023513D4F4C2F6091EA020E945519F394B7
:103A2000E3CF0E94D419F8018481811102C091E092
:103A300003C0803219F49FEF9093250190912501E6
:103A4000890FF8018483DF91CF911F910F91FF902F
:103A5000EF90DF90CF90BF90AF909F908F900895A0
:103A60000F931F93CF93DF93EC0100E010E0809160
:103A70002C01282F30E00217130724F590912A011A
:103A80009801290F311DA901440F551F240F351F1F
:103A900023513D4F869590E04C81081719071CF47F
:103AA000442331F002C0411103C04091EB0201C038
:103AB00040E06091EA028091E9020E9455190F5F8F
:103AC0001F4FD5CF0E94D4198C8190E00196817050
:103AD00099278C83DF91CF911F910F910895E8EE84
:103AE000F2E080818E7F8083608171818281938109
:103AF0000E947A191092AD022FEF80E792E02150D8
:103B000080409040E1F700C000000C94D41960910F
:103B1000E802669570E04BE050E08DE291E00E9493
:103B2000942E892B19F481E08093AD020E94F51147
:103B30009093A6028093A50208959091E80290FFC9
:103B400035C09170811102C0926006C0853210F0BC
:103B5000986402C0880F982B9093E802662351F076
:103B60006091E8027091E9028091EA029091EB0283
:103B70000E947A196091E802669570E04BE050E08F
:103B80008DE291E00E94942E892B19F01092AD02E3
:103B900002C00E94871D81E08093A8024091EB0241
:103BA0006091EA028091E9020C94781B0895682FD5
:103BB0009091E802969581E0890F853208F081E0C6
:103BC0000C949D1D81E00C94D71D682F9091E80204
:103BD00096958FEF890F09F484E20C949D1D81E086
:103BE0000C94E51D61E00C949D1DE8EEF2E08081EF
:103BF0008160808386950C94F21D8091E80280FD9F
:103C00000C946F1D0C94F51D60E00C949D1D80912B
:103C1000AB0281112EC00E94220E811104C00E94AD
:103C2000CF0E0E948C190E9476196093E80270935F
:103C3000E9028093EA029093EB026E7F61F40E94A6
:103C40008C190E9476196093E8027093E9028093C0
:103C5000EA029093EB020E9463191092AD028091E8
:103C6000E80280FF03C086950E94041E81E08093D5
:103C7000AB0208950F931F93CF93DF938091AD0212
:103C8000882309F485C08091AC02E091E802E695B2
:103C9000E81BE093A702823049F4F0E0E250FE4FC7
:103CA000E491CE2FD0E00DE21AE149C0863049F40C
:103CB000F0E0E550FE4FE491CE2FD0E001E41AE1B0
:103CC0003EC0893051F4E695F0E0E850FE4FE491B3
:103CD000CE2FD0E00BE71BE132C08F3051F4E695D8
:103CE000F0E0EB50FE4FE491CE2FD0E006EB1BE16D
:103CF00026C0853149F4F0E0EE50FE4FE491CE2F1E
:103D0000D0E00BE21CE11BC0883181F0833239F432
:103D1000E0EFF1E0C591D49101E51AE110C08432E1
:103D200051F4C4EFD1E000E31DE109C0C8E2D0E0E6
:103D30000DE91CE104C0C0EDD7E001E519E1809177
:103D4000A802882361F01092A8020E94F5119093B6
:103D5000A6028093A5021092AA021092A9020E94C4
:103D6000F511E091A502F091A6028E1B9F0B8F3FEB
:103D70009F4770F4EC0FFD1FF093A602E093A5029D
:103D800085EA92E0F801DF91CF911F910F9109949C
:103D9000DF91CF911F910F910895882311F0FA01BF
:103DA00001C0FB010994CF93DF93C82FD62F0E9447
:103DB0009B198C1740F00E949B198D1720F4DF91FE
:103DC000CF910C94E21D8C2FDF91CF910C94F21DBA
:103DD0001F93CF93DF93FB0112811111C3C0EC013C
:103DE0000E943F0D8272CD3CFCE5DF0709F49AC0CA
:103DF000A8F5C73CECE5DE0709F476C0A8F4C43C9E
:103E00009CE5D90709F45FC028F4C33CDC4509F4FC
:103E100057C054C0C53C9CE5D90709F459C0C63CFD
:103E2000DC4509F45CC04AC0CA3CFCE5DF0709F484
:103E30006AC050F4C83CECE5DE0709F45AC0C93C3E
:103E4000DC4509F45BC03AC0CB3C9CE5D90709F4DA
:103E50005FC0CC3CDC4509F460C030C0C23DFCE52D
:103E6000DF0709F46FC088F4CF3C9CE5D90709F45B
:103E700060C008F45CC0C03DFCE5DF0709F45CC02D
:103E8000C13DDC4509F45BC019C0C53D9CE5D907BF
:103E900009F460C050F4C33DFCE5DF0709F455C0E8
:103EA000C43DDC4509F454C009C0C63D9CE5D907B2
:103EB00009F455C0CE35DD4509F454C011E052C0B7
:103EC0000E94FD1D4FC04FEE5DE162EE7DE104C03A
:103ED00042EE5DE16FEE7DE10E94CD1E43C049E3FD
:103EE0005BE16CE27BE1F8CF4CE25BE169E37BE113
:103EF000F3CF47E55BE168E47BE1EECF48E45BE1CB
:103F000067E57BE1E9CF45E75BE166E67BE1E4CF8E
:103F100046E65BE165E77BE1DFCF4EEC59E167EB1D
:103F200079E1DACF47EB59E16EEC79E1D5CF81E069
:103F300017C065E082E010C068E086E00DC06EE06A
:103F400089E00AC064E18FE007C067E185E104C051
:103F500088E106C062E289E10E94D31E03C083E2C9
:103F60000E94F21D812FDF91CF911F910895519AE8
:103F70002BB12D7F3BB132604FB7F894FC01CB01E0
:103F8000880F991F680F791F6E0F7F1FE617F707BD
:103F900089F0819198E03BB9000000C087FF2BB900
:103FA000880F000000C000C000C02BB900C09A9567
:103FB00091F7ECCF4FBF8FE594E00197F1F700C088
:103FC000000008950895FC01680F791F8FEF91E3B9
:103FD000E617F70771F02191822728E030E087FF8C
:103FE00003C0880F892701C0880F21503109B9F714
:103FF000EFCF0895CF93DF93EC01FB0182818823FB
:1040000009F43CC1C430FDE5DF0760F4CB3F9CE51B
:10401000D90788F49E0122503C452431310508F02F
:104020002EC109C0C236EDE5DE0729F0C63AFDE52E
:10403000DF0709F024C10E943A0E9093D1028093C9
:10404000D002C1318CE5D80709F4C6C008F042C0DF
:10405000C930ECE5DE0709F49BC000F5C5308CE5FE
:10406000D80709F485C078F4C330ECE5DE0709F41D
:1040700078C008F07AC0C230DC4509F0F5C0809104
:10408000D0028160EFC0C7309CE5D90709F478C041
:1040900008F07AC08091D0028061E4C0CD30FCE5A8
:1040A000DF0709F487C058F4CB309CE5D90709F441
:1040B00079C008F07BC08091D00288606FC0CF309B
:1040C000FCE5DF0709F480C008F082C08091D002CF
:1040D000877FC8C0CE3F9CE5D90709F471C000F5C1
:1040E000C531FCE5DF0709F485C068F4C3319CE500
:1040F000D90709F475C008F095C00E94EC078091BB
:10410000D0028F77AFC0CC3FFCE5DF07A9F108F004
:1041100054C0CB3FDC4509F0A7C08091D10240C01C
:10412000C230EDE5DE0709F489C058F4C1158DE50C
:10413000D80709F45AC008F069C08091D1028260A2
:104140002FC0C236EDE5DE0709F47CC0C63AFDE5B6
:10415000DF0709F481C0C330DD4509F085C080E088
:104160006EC08091D00282607DC08091D00216C066
:104170008091D002886076C08091D10282604FC069
:104180008091D00280626EC08091D00280646AC04B
:104190000E94EC078091D002806864C0846062C095
:1041A00081603DC08091D0028E7F5CC08091D00242
:1041B0008D7F58C08091D00216C08091D10218C066
:1041C0008091D1028D7F2BC08091D0028F7E4AC01A
:1041D0008091D0028F7D46C08091D0028F7B42C0FB
:1041E0008091D002877F8B7F3DC08091D1028D7FEF
:1041F0008E7F15C08091D00282FB222720F991E0AA
:10420000922790FB82F990FB83F92CC08091D10218
:10421000982F909591708E7F892B90FB81F98093D8
:10422000D10222C00E94EC078091D00287FB222796
:1042300020F991E0922790FB87F914C081E00E9459
:10424000D10E12C08091D00284FB222720F991E088
:10425000922790FB84F906C08091D002982F909508
:1042600090FB80F98093D0028091D0029091D1028E
:104270000E944B0E0E94EC0780E001C081E0DF91BC
:10428000CF910895893289F1F0F4843171F1B0F45D
:10429000873009F077C081E08093240184E1809326
:1042A00023018AE0809322018EE18093210188E03E
:1042B00080931E0188E280931D0164C092EE980FE6
:1042C0009A30F0F05FC0803509F444C028F48F3490
:1042D00009F058C08AE03FC0813529F0823509F0E5
:1042E00051C081E038C08FEF36C08091B002882382
:1042F00079F11092B0021092AF021092AE0242C059
:104300008D518093B002833099F038F4813069F098
:104310008230D9F483E291E00DC0853099F078F0D5
:10432000863099F48DE191E005C084E291E002C00D
:1043300082E291E09093AF028093AE0223C081E2CB
:1043400091E0F8CF8EE191E0F5CF1092B0021AC063
:1043500080E0089586EFE091AE02F091AF023097D1
:1043600089F02081082E000C990B820F911D8F3F40
:10437000910519F014F08FEF04C097FF02C010826E
:1043800001C0808381E008950F931F9341E050E0C6
:1043900060E070E08A019B0104C0000F111F221F22
:1043A000331F8A95D2F7C901B8010E9444081F91B2
:1043B0000F910C94EC078B3109F468C058F58B30E1
:1043C00009F486C078F4863009F445C020F48530BD
:1043D00009F44BC07FC0873009F44AC0883009F423
:1043E00077C078C0803109F464C068F48E3009F079
:1043F00071C08091710282FB222720F991E09227FF
:1044000090FB82F94CC0863109F462C0893109F40D
:104410005FC060C08A32E1F060F4873209F455C0B1
:1044200028F48E3108F456C08D5150C08932E9F01D
:1044300051C0833450F48A3308F045C0853309F401
:1044400044C0883309F444C045C08334F1F142C00C
:104450000E94CF0E3DC080917102817F8E7F80933C
:10446000710281E08093B10208950E942F0330C051
:1044700080917102982F9095917090FB80F98093B4
:104480007102911125C0897F877F10C080917102D0
:1044900081FB222720F991E0922790FB81F98093FC
:1044A00071029923A9F08091710281608093710259
:1044B0000FC08091710283FB222720F991E092279F
:1044C00090FB83F9ECCF895301C080E00E94C421A6
:1044D00081E0089580E0089580E008950C946C22B6
:1044E000CF93C82F8091B102813069F038F08230CB
:1044F000C1F58C2F0E94422181E039C00E943F0DFE
:10450000823289F504C00E943F0D823261F48C2F03
:104510000E946E22811104C08C2F0E94DB211FC0DB
:1045200081E090E01CC08C2F0E946C22811116C08B
:10453000C43189F058F4CB3089F0C031B1F482E055
:104540008093B10288E30E94422108C0C93219F069
:10455000C83321F00AC01092B10207C081E0817017
:1045600006C01092B10280E002C080E0F8CFCF9187
:104570000895CF93DF9386319C4541F5EB010E946E
:104580003F0D982F8A8120910201309103018823E9
:1045900079F09A7A81E009F480E08093B202911177
:1045A00002C069E201C065E3C9010E9415260AC084
:1045B0008091B202811102C069E201C065E3C901C4
:1045C0000E9417260E94810D80E001C081E0DF91EA
:1045D000CF9108950F931F93CF93DF93C42FD22FC2
:1045E000FC0182818823C9F04093B5020E94BB265A
:1045F0009093B4028093B30280E28C0F883008F06D
:1046000057C0C77081E001C0880FCA95EAF7DF91F3
:10461000CF911F910F910C9449058091B5024813D9
:1046200030C08091B3029091B4020E94D326883C9E
:10463000910538F510E21D0FCD17B9F080E28C0F0F
:10464000883040F4C77081E001C0880FCA95EAF74E
:104650000E945005183028F581E09D2F977001C009
:10466000880F9A95EAF70E944905802F0E9440051D
:104670001830F0F4D77081E001C0880FDA95EAF7BE
:104680000AC080E28C0F883098F4C77081E001C0C6
:10469000880FCA95EAF7DF91CF911F910F910C9483
:1046A0005005802FDF91CF911F910F910C94400501
:1046B000DF91CF911F910F9108950F939C01CB0132
:1046C000243F4CE5340731F188F4293DFCE53F07F0
:1046D000D9F02A3D4CE5340779F1283D3C45A9F550
:1046E00006E221EE41EE68ED7CE52BC0263FFCE5BD
:1046F0003F07E1F0A8F0273F3C4539F507E225EEFA
:1047000046EE67EF7CE51DC007E225EE45EE69ED5C
:104710007CE517C006E221EE40EE64EF7CE511C0B7
:1047200007E225EE44EE65EF7CE50BC006E221EEE4
:1047300042EE66EF7CE505C008E221E045EE6AED59
:104740007CE50E94EA2280E008C0FC018281882387
:1047500019F01092B50201C081E00F9108958EE129
:10476000489B02C08150E1F7489BFECF08955898BE
:1047700080E28A95F1F7589A0895FC012AE02A957B
:10478000F1F728E090E080E031E040E14A95F1F770
:10479000880F489B02C08160932700C0000040E161
:1047A0004A95F1F7215089F720E12A95F1F729B1CF
:1047B00000C0000030E13A95F1F721709227208186
:1047C000920F90830895EF92FF920F931F93CF93D0
:1047D000DF931F92CDB7DEB719828C017C01E60E04
:1047E000F11C0E151F0551F00E94AF23CE0101965A
:1047F0000E94BD23F80181938F01F3CF81E099815D
:10480000911180E00F90DF91CF911F910F91FF9058
:10481000EF900895509A589A08955098589AE89AA7
:10482000E9E6F0E080818C7F80830895615091E01B
:1048300001C0990F6A95EAF720E031E0992361F011
:10484000492F482319F0589A232701C0589840E26D
:104850004A95F1F79695F2CF222311F0589A01C0AC
:10486000589880E28A95F1F758980895FF920F932F
:104870001F93CF93DF93EC018C01060F111DC0171E
:10488000D10741F0F9900E94B72368E08F2D0E9474
:104890001624F5CFDF91CF911F910F91FF900895CE
:1048A0001F920F920FB60F9211240F931F932F9305
:1048B0003F934F935F936F937F938F939F93AF93A8
:1048C000BF93EF93FF93CF93DF931F92CDB7DEB7E4
:1048D00019820E94AF23CE0101960E94BD23082FAA
:1048E000069506950695902F96959570202F257024
:1048F000920F292F237096959695920F87708913A2
:104900005FC0898181115CC0043008F059C080E12A
:104910008A95F1F7589A509A82E08A95F1F700C08B
:10492000589888E0089F80011124D801AB5FBE4FE2
:104930001696ED91FC9117973097A9F06091B3010D
:104940007091B40114962D913C911597260F371F45
:1049500011968D919C911297680F791F13964C9127
:1049600013978C910995F801EB5FFE4F63816623E5
:1049700051F08091B3019091B40124813581820F6F
:10498000931F0E9436240E94B72380E18A95F1F795
:1049900058985098589A80E18A95F1F7F801EB5FA2
:1049A000FE4F6081662351F08091B3019091B40174
:1049B00021813281820F931F0E94E3230E94AF2343
:1049C0000F90DF91CF91FF91EF91BF91AF919F91A8
:1049D0008F917F916F915F914F913F912F911F9197
:1049E0000F910F900FBE0F901F9018950F931F936C
:1049F000CF93DF93843091050CF06DC0EC01F894F7
:104A0000509A589885E08A95F1F700009C2F96956A
:104A100095702C2F2570920F892F837096959695FF
:104A200023E0CC0FDD1F2A95E1F7980F8E01092BAB
:104A30000E94B72384E08A95F1F700C068E0802FD8
:104A40000E94162480E18A95F1F75098589A489967
:104A500002C000C0FCCF87E090E0489B08C00197EF
:104A600021F4509A589A789436C000C0F6CFFE01CF
:104A7000EB5FFE4F6381662381F08091B3019091DB
:104A8000B40124813581820F931F0E94E323811199
:104A900004C0509A589A78941FC00E94AF2380E2B5
:104AA0008A95F1F75898509A80E18A95F1F7CB5F93
:104AB000DE4F6881662351F08091B3019091B4017B
:104AC00029813A81820F931F0E9436240E94B723C6
:104AD000789481E001C080E0DF91CF911F910F9128
:104AE00008959093DB018093DA0108959093BC02BE
:104AF0008093BB0208950E94EF13811103C080913F
:104B0000B6020895E091BB02F091BC02309721F00B
:104B10000190F081E02D099480E00895E091BB02BE
:104B2000F091BC02309721F00280F381E02D0994CE
:104B30000895E091BB02F091BC02309739F022E079
:104B4000DC012C930480F581E02D099408952091D7
:104B5000B9023091BA022817390771F09093BA025E
:104B60008093B902E091BB02F091BC02309721F032
:104B70000680F781E02D099408952091B7023091C5
:104B8000B8022817390771F09093B8028093B702E2
:104B9000E091BB02F091BC02309721F00084F185D6
:104BA000E02D09940895FC01329697E080E0915041
:104BB00029F021912223D9F38F5FF9CF089566233D
:104BC00049F0FC01329608962191621729F0E81706
:104BD000F907D1F780E0089581E008959C01FC0178
:104BE00032969FEF80E04191461789F09F3F19F47C
:104BF000411101C0982F8F5F8630A9F79F3F39F090
:104C0000F901E90FF11D97FDFA9562830895089562
:104C10009C012A5F3F4FFC014281461301C0128272
:104C2000019682179307B9F708950C94EE250C941A
:104C30000826029626E0FC0111922A95E9F70895CC
:104C400008950C94202683E08093BD020C942126C5
:104C5000811102C081E001C082E08093BD020C940A
:104C600021260C94282681E08093BD020C942126F5
:104C70000C94332608950C943A260C943B260C94FD
:104C80003A260C943A260C943A26CF930E94412659
:104C90000E9464130E943F26C0E08C2F0E942512C0
:104CA000811104C0CF5FCA30C1F701C081E0CF914C
:104CB000089508951F920F920FB60F9211248F93AB
:104CC0009F93AF93BF938091BE02811113C08091D7
:104CD0001D0390911E03A0911F03B09120034196E4
:104CE000A11DB11D80931D0390931E03A0931F036C
:104CF000B0932003BF91AF919F918F910F900FBE02
:104D00000F901F90189580912503843031F10E94F7
:104D100097031092BE0220E488E190E00FB6F89469
:104D2000A895809360000FBE2093600083B7817FB9
:104D3000846083BF83B7816083BF7894889583B78D
:104D40008E7F83BF0FB6F894A8958091600088612C
:104D500080936000109260000FBE08950E94EC07DF
:104D60000C949B0382E084BD93E095BD9AEF97BDC0
:104D700080936E0008952FB7F89480911D03909151
:104D80001E03A0911F03B09120032FBF08952FB7DA
:104D9000F89460911D0370911E0380911F03909100
:104DA00020032FBF08959C014FB7F89480911D03F5
:104DB00090911E03A0911F03B09120034FBF821B4F
:104DC000930B0895CF92DF92EF92FF922FB7F89452
:104DD000C0901D03D0901E03E0901F03F0902003AD
:104DE0002FBFA7019601261B370B480B590BCA0191
:104DF000B901FF90EF90DF90CF90089578941F92C3
:104E00000F920FB60F9211248F939F93AF93BF937E
:104E100080911D0390911E03A0911F03B091200368
:104E20000196A11DB11D80931D0390931E03A093B5
:104E30001F03B0932003BF91AF919F918F910F906B
:104E40000FBE0F901F90189587E797E79093010882
:104E5000809300089AE088E10FB6F894A8958093B3
:104E600060000FBE90936000FFCF8091CA0208954A
:104E7000089522E02093E9002FEF3091E8002150BF
:104E800035FD06C035ED3A95F1F700002111F5CF5B
:104E90002091E80025FF0BC040E050E066E070E0A4
:104EA0000E9463298091E8008E778093E80008953E
:104EB000CF93DF9321E02093E9002FEF3091E800BA
:104EC000215035FD06C035ED3A95F1F7000021116E
:104ED000F5CF2091E80025FF14C0EC0140E050E040
:104EE00068E070E00E9463298091E8008E778093EB
:104EF000E80088E0FE01A2ECB2E001900D928A95F4
:104F0000E1F7DF91CF9108958093BF027093C102C2
:104F10006093C00280912503843001F582E0809384
:104F2000E9008FEF9091E800815095FD06C095ED66
:104F30009A95F1F700008111F5CF8091E80085FF87
:104F40000DC040E050E063E070E08FEB92E00E9423
:104F500063298091E8008E778093E8000895BC0172
:104F600084E00C948427BC0183E00C948427809116
:104F70002403811109C00E94F42A0E94512B8091C0
:104F8000E20084608093E200089510922403089563
:104F90000C9438266091210381E0611101C080E00A
:104FA0000C9423269091250381E0943009F080E051
:104FB000609121030C94282642E061EC81E00E947C
:104FC0006D2A42E261EC82E00E946D2A90912503F5
:104FD00081E0943009F080E0609121030C94312647
:104FE00080912703833009F461C030F4813071F07F
:104FF000823009F49AC008958A3009F486C08B3053
:1050000009F46CC0893009F0A8C020C08091260343
:10501000813A09F0A2C08091E800877F8093E80080
:1050200080912A0390912B03892B21F468E082EC74
:1050300092E003C060E080E090E070E00E94AE2962
:105040008091E8008B778093E80008958091260393
:10505000813209F082C080912A0390912B0302973C
:1050600008F07BC08091E800877F8093E800809102
:10507000E80082FD05C0809125038111F8CF6DC045
:105080002091F3008091F20090E0922B029731F48E
:105090008091F100813011F0863021F48091F1008F
:1050A0008093CA028091E8008B7753C080912603D9
:1050B000813A09F052C080912A0390912B03892BE9
:1050C00009F04BC08091E800877F8093E8008091D1
:1050D000E80080FFFCCF8091440136C08091260318
:1050E0008132D9F580912A0390912B03892BA9F560
:1050F0008091E800877F8093E8000E94A22A809137
:105100002803809344010C94EC078091260381329C
:1051100021F58091E800877F8093E8000E94A22A11
:10512000809129038093CB02089580912603813AD0
:10513000A1F48091E800877F8093E8008091E800E7
:1051400080FFFCCF8091CB028093F1008091E8003A
:105150008E778093E8000C94A22A089584B7877F05
:1051600084BF0FB6F894A895809160008861809301
:105170006000109260000FBE90E080E80FB6F894D7
:1051800080936100909361000FBE0C9433260E94BF
:10519000F42A0E94512BE2EEF0E08081846080834B
:1051A00078940C94E62D88E391E00C947625809118
:1051B00025038530A9F480912503853079F40E9478
:1051C0008326809123038823B1F30E9445268823F8
:1051D00091F30E944D290E94EC07EDCF0C94AE266E
:1051E000089508950C94F428292F3327233031058E
:1051F000C9F060F42130310581F02230310509F029
:1052000044C08BE390E027E334E043C02132310512
:10521000E1F02232310549F138C082E190E022E725
:1052200034E037C099278130910549F028F0029782
:1052300061F5E7E0F4E005C0E3E3F4E002C0E1E299
:10524000F4E0849190E09F0124C06115710541F064
:1052500061307105D1F489E090E022E634E019C0B4
:1052600089E090E029E434E014C06115710541F053
:105270006130710551F48BE790E024E834E009C017
:1052800080E490E02FEF34E004C080E090E020E084
:1052900030E0FA0131832083089580E189BD82E105
:1052A00089BD09B400FEFDCF8091D8008F7D809329
:1052B000D8008091E00082608093E0008091E0005F
:1052C00081FDFCCF0895CF92DF92EF92FF920F9372
:1052D0001F93CF93DF93EC018B017A010E94C12AC7
:1052E000811133C0E114F10439F0F701808191811B
:1052F000081B190BC80FD91FC12CD12C0115110582
:1053000019F18091E80085FD16C08091E8008E7744
:105310008093E800E114F10449F0F7018081918164
:10532000C80ED91ED182C08285E00FC00E94C12A5A
:10533000882321F30AC089918093F100015011095B
:10534000FFEFCF1ADF0ADACF80E0DF91CF911F9114
:105350000F91FF90EF90DF90CF90089520912C0354
:1053600030912D032617370748F06115710539F480
:105370002091E8002E772093E80001C0B901FC01DC
:1053800020E06115710579F1809125038823F1F101
:105390008530F1F18091E80083FD3CC08091E80008
:1053A00082FD2EC08091E80080FFEBCF2091F300BA
:1053B0008091F20090E0922B6115710551F08830D8
:1053C000910538F421912093F10061507109019603
:1053D000F3CF21E0089709F020E08091E8008E7774
:1053E0008093E800CECF2111CFCF0AC08091250352
:1053F000882361F0853061F08091E80083FD0AC068
:105400008091E80082FFF2CF80E0089582E0089565
:1054100083E0089581E0089520912C0330912D03BD
:105420002617370748F06115710539F42091E80017
:105430002E772093E80001C0B901FC0120E061153E
:10544000710591F180912503882309F440C08530CE
:1054500009F43FC08091E80083FD3DC08091E800E1
:1054600082FD2FC08091E80080FFE9CF2091F300FA
:105470008091F20090E0922B6115710559F088300F
:10548000910540F424912093F10031966150710907
:105490000196F2CF21E0089709F020E08091E80022
:1054A0008E778093E800CBCF2111CCCF0AC08091BA
:1054B0002503882361F0853061F08091E80083FD49
:1054C0000AC08091E80082FFF2CF80E0089582E078
:1054D000089583E0089581E00895982F973068F546
:1054E0009093E900981739F07091EC002091ED004D
:1054F0005091F00003C0242F762F50E021FD02C010
:105500009F5FECCF3091EB003E7F3093EB0030910A
:10551000ED003D7F3093ED003091EB003160309332
:10552000EB007093EC002093ED005093F00020917D
:10553000EE0027FDE5CF80E008958F708093E900AD
:1055400081E008958091260387FF11C08091E800D3
:1055500082FD05C0809125038111F8CF11C0809193
:10556000E8008B770BC080912503882349F0809158
:10557000E80080FFF8CF8091E8008E778093E80004
:1055800008952091E4003091E50095E64091EC000B
:10559000842F817040FF23C08091E80080FD1DC0F2
:1055A00080912503882399F0853099F08091EB0054
:1055B00085FD11C04091E4005091E50024173507A6
:1055C00029F3915011F09A01E1CF84E0089582E02F
:1055D000089583E0089581E0089580E00895409162
:1055E000E80042FFDDCF08950E94622B0E946A2BE3
:1055F000E0EEF0E0808181608083E8EDF0E0808182
:105600008F77808319BCA7EDB0E08C918E7F8C934F
:1056100080818F7E80831092240308950F931F93BF
:10562000CF93DF930E94622B0E946A2BC8EDD0E0DB
:1056300088818F77888388818068888388818F7D3F
:10564000888319BC10922503109221031092230322
:105650001092220300EE10E0F80180818B7F80839E
:1056600088818160888342E060E080E00E946D2A4A
:10567000E1EEF0E080818E7F8083E2EEF0E08081D9
:1056800081608083808188608083F80180818E7F43
:105690008083888180618883DF91CF911F910F91F2
:1056A0000895E8EDF0E080818F7E8083E7EDF0E003
:1056B00080818160808384E082BF81E080932403C5
:1056C0000C940E2BE8EDF0E080818E7F80831092A9
:1056D000E20008951092DA001092E10008951F92FE
:1056E0000F920FB60F9211242F933F934F935F9316
:1056F0006F937F938F939F93AF93BF93EF93FF939A
:105700008091E10082FF0BC08091E20082FF07C020
:105710008091E1008B7F8093E1000E94E52D8091D4
:10572000DA0080FF1FC08091D80080FF1BC08091ED
:10573000DA008E7F8093DA008091D90080FF0DC05F
:1057400080E189BD82E189BD09B400FEFDCF81E021
:10575000809325030E94B72705C019BC109225032A
:105760000E94C5278091E10080FF19C08091E2006E
:1057700080FF15C08091E2008E7F8093E2008091CF
:10578000E20080618093E2008091D8008062809383
:10579000D80019BC85E0809325030E94CA27809118
:1057A000E10084FF30C08091E20084FF2CC080E1E2
:1057B00089BD82E189BD09B400FEFDCF8091D8008A
:1057C0008F7D8093D8008091E1008F7E8093E100EF
:1057D0008091E2008F7E8093E2008091E200816000
:1057E0008093E20080912103882311F084E007C0B8
:1057F0008091E30087FD02C081E001C083E08093D7
:1058000025030E94D2278091E10083FF29C0809167
:10581000E20083FF25C08091E100877F8093E10053
:1058200082E080932503109221038091E1008E7F16
:105830008093E1008091E2008E7F8093E20080916E
:10584000E20080618093E20042E060E080E00E943C
:105850006D2A8091F00088608093F0000E94C82734
:10586000FF91EF91BF91AF919F918F917F916F9138
:105870005F914F913F912F910F900FBE0F901F900E
:1058800018951F920F920FB60F9211242F933F93EA
:105890004F935F936F937F938F939F93AF93BF9338
:1058A000CF93DF93EF93FF93C091E900CF70809186
:1058B000EC00D82FD17080FDD0E81092E9008091E3
:1058C000F000877F8093F00078940E94852C1092DE
:1058D000E9008091F00088608093F000CD2BCF70BC
:1058E000C093E900FF91EF91DF91CF91BF91AF910C
:1058F0009F918F917F916F915F914F913F912F91E8
:105900000F900FBE0F901F9018951F93CF93DF93AA
:10591000CDB7DEB7AA970FB6F894DEBF0FBECDBFE6
:10592000E6E2F3E08091F100819323E0EE32F207AA
:10593000C9F70E94F0278091E80083FF2EC1809173
:10594000260390912703492F50E04A30510508F073
:1059500024C1FA01EE59FF4F0C945D2E803821F0DE
:10596000823809F01AC108C0809122039091230364
:10597000992389F082600FC080912A038F7087304D
:1059800008F00BC18093E9008091EB0085FB88272C
:1059900080F91092E9009091E800977F9093E800D9
:1059A0008093F1001092F100D1C0282F2D7F09F0D3
:1059B000F4C0882319F0823061F0EFC08091280391
:1059C000813009F0EAC0933009F080E0809323032E
:1059D0002EC08091280381112AC080912A038F70E4
:1059E0002FEF280F263008F0D8C08093E9002091CF
:1059F000EB0020FF1CC0933021F48091EB0080620B
:105A000014C09091EB0090619093EB0021E030E0A6
:105A1000A90102C0440F551F8A95E2F74093EA009E
:105A20001092EA008091EB0088608093EB00109266
:105A3000E9008091E800877F8093E8000E94A22A15
:105A4000ACC08111AAC0109128031F778091E30098
:105A50008078812B8093E3008091E800877F80939A
:105A6000E8000E94A22A8091E80080FFFCCF80918C
:105A7000E30080688093E300111102C082E001C05E
:105A800083E08093250389C08058823008F085C068
:105A900080912803909129038C3D53E0950779F577
:105AA00083E08A838AE289834FB7F894DE011396F4
:105AB00020E03EE051E2E32FF0E050935700E49104
:105AC00020FF03C0E295EF703F5FEF708E2F90E0F4
:105AD000EA3010F0C79601C0C0968D939D932F5F5A
:105AE000243149F74FBF8091E800877F8093E80019
:105AF0006AE270E0CE0101960E94AE2916C0609164
:105B00002A0370912B03AE014F5F5F4F0E94F22872
:105B1000BC01892B09F441C09091E800977F9093D4
:105B2000E80089819A810E940C2A8091E8008B7795
:105B30008093E80032C0803881F58091E800877F4B
:105B40008093E800809121038093F1008091E80028
:105B50008E7772CF811121C0809128039091290303
:105B600099270297D4F48091E800877F8093E8001A
:105B700080912803809321030E94A22A809121030F
:105B8000811106C08091E30087FD02C081E001C061
:105B900084E0809325030E94DC278091E80083FF46
:105BA0000AC08091E800877F8093E8008091EB0035
:105BB00080628093EB00AA960FB6F894DEBF0FBE0A
:105BC000CDBFDF91CF911F9108950895CF9380911C
:105BD00025038823A1F0C091E900CF709091EC00DB
:105BE000892F817090FD80E8C82B1092E900809188
:105BF000E80083FD0E94852CCF70C093E900CF910F
:105C000008950E94F42A109225030895E8EDF0E02B
:105C10008081806180838AE18A95F1F700C080915C
:105C2000D90081700895AA1BBB1B51E107C0AA1FB0
:105C3000BB1FA617B70710F0A61BB70B881F991F2D
:105C40005A95A9F780959095BC01CD01089597FBD1
:105C5000072E16F4009407D077FD09D00E94132E6A
:105C600007FC05D03EF4909581959F4F089570955F
:105C700061957F4F0895A1E21A2EAA1BBB1BFD015F
:105C80000DC0AA1FBB1FEE1FFF1FA217B307E4071B
:105C9000F50720F0A21BB30BE40BF50B661F771F73
:105CA000881F991F1A9469F7609570958095909553
:105CB0009B01AC01BD01CF010895EE0FFF1F0590C0
:105CC000F491E02D09940E946B2E332312F48A1B69
:105CD0009B0B0C947C2EA29FB001B39FC001A39F8D
:105CE000700D811D1124911DB29F700D811D112415
:105CF000911D08950E946B2EB7FF0895821B930B90
:105D000008950E946B2EA59F900DB49F900DA49FA7
:105D1000800D911D11240895B7FF0C94812E0E94CF
:105D2000812E821B930B0895FC014150504030F0AE
:105D300001900616D1F73197CF010895882799274A
:105D40000895FB01DC0104C08D910190801921F4BC
:105D500041505040C8F7881B990B0895FB01DC01A6
:105D600002C001900D9241505040D8F70895F99922
:105D7000FECF92BD81BDF89A992780B50895A6E11E
:105D8000B0E044E050E00C94F12EA8E1B0E042E035
:105D900050E00C94F12E262FF999FECF92BD81BDD3
:105DA000F89A019700B4021639F01FBA20BD0FB659
:105DB000F894FA9AF99A0FBE08950396272F0E9435
:105DC000CC2E0E94CB2E252F0E94CC2E242F0C945B
:105DD000CC2E0196272F0E94CC2E0C94CB2EDC01CA
:105DE000CB01FC01F999FECF06C0F2BDE1BDF89AE6
:105DF000319600B40D9241505040B8F70895F89490
:025E0000FFCFD2
:105E0200C80055020100000001000000000000006F
:105E120005010000000406000000000000280850F0
:105E2200011E0A1401010102001000101001191ACA
:105E32001B1C1D1E1F202122352758273927B32757
:105E4200AF27382701E200E900EA00B500B600B743
:105E520000CD008301CC008A01920194012102232A
:105E62000224022502260227022A02B300B4006F8E
:105E7200007000818283E200E900EA00B500B6000A
:105E8200B700CD008301CC008A0192019401210266
:105E9200230224022502260227022A02B300B400AA
:105EA2006F007000818283323331F7F69436669741
:105EB200C634357A02000102020202060606090908
:105EC200090909090F0F0F0F0F0F151515181919C9
:0A5ED20019191919191919192324B7
:00000001FF
